:10000000EFEF03F000000000E4EF03F00000000059
:0A0010000000000000000000F3D71C
:10001C00026A036A800E0318006E800E005C02E117
:10002C00080E025C11E28296800E01016215016ECF
:10003C000150800A02E1828801D082988286623760
:0A004C006291024A032AE6D712006F
:100056008292829061C162F1DEDF070E0C6E7D0E28
:0E0066000D6E0D2EFED70C2EFCD782801200E0
:10007400070E01016015006E400E0010616FE9DF8C
:100084007F0E01015F15006E800E0010616FE1DFCD
:02009400120058
:0E009600828282905FC162F1BEDF8280120022
:1000A4008194040E0C6E3D0E0D6E0D2EFED70C2E9B
:1000B400FCD700000000010E036E800E080A006EDB
:1000C400800E0318005C19E3819A800E01015A1511
:1000D400016E000E5ABFFF0E026E000E0216000ED5
:1000E400021802E1800E011802E1818001D08190A2
:1000F4005A375A91818A032AE0D78184818A12006F
:10010400200E01015A5D04E35A517F0801E301D036
:100114001200050E5A03F3CF00F0F4CF01F0A00E45
:10012400005C5B6F000E01585C6F050E5D6F000E86
:100134005E6F800E006E800E5E19005C02E15D5100
:10014400000818E25C0E5B25F66E0D0E5C21F76E5E
:10015400000EF86E000E5CBFFF0EF8220900F5CF0A
:100164005FF197DF01015B4B5C2B010E5D5F000EBD
:0A0174005E5BDFD75F6B8DDF1200CA
:10017E00086A096A100E0C6E0134083609360450EE
:10018E00085E0550D8A0053C095ED8B007D00450D3
:10019E0008260550D8B0053C0926D8900036013601
:0601AE000C2EEAD712003E
:1001B4008194040E0C6E3D0E0D6E0D2EFED70C2E8A
:1001C400FCD700000000056A066A076A086A0F0E79
:1001D400046E800E0418006E800E000A005C24E396
:1001E400819A818A81A81ED00404006E000E04BE88
:1001F400FF0E016E000E015A00C002F0010E006EE7
:10020400000E016E025005E0003600900136FF0F2B
:10021400FAD70050052601500622000E01BEFF0E3B
:10022400072208220406D5D7818405C000F006C041
:0C02340001F007C002F008C003F0120047
:100240005AC102F05BC103F002C000F003C001F02C
:10025000024A032A00C0E9FF01C0EAFFEE5201E0B2
:10026000F3D701015A51025C006E5B510358016ED5
:0A027000010E005E000E015A12009C
:0E027A00ACB202D00000FCD75AC1ADFF12009A
:10028800086A080E0C6E003408360450085ED8B0B0
:0E02980002D00826D89000360C2EF5D71200A2
:1002A60001015F6B606BE3DE01015A6B5B6B800ED5
:1002B600030A006E800E5B19005C02E15A51800849
:1002C60010E35F6BE5DE040E0C6E3D0E0D6E0D2E1B
:1002D600FED70C2EFCD70000000001015A4B5B2B09
:0402E600E6D7120045
:1002EA000101576B050E575D0AE257515525E16E1C
:1002FA00000E5621E26E200EE66E572BF3D75751A9
:10030A005525E16E000E5621E26EE66A57075751EF
:10031A005525586F000E5621596F0A0E046E000EAD
:10032A00056E53C100F054C101F024DF08C000F08B
:10033A0009C001F0300E002658C1E1FF59C1E2FFA1
:10034A0000C0E6FF0A0E046E000E056E53C100F0EF
:10035A0054C101F00FDF00C053F101C054F1000E87
:10036A00011802E1000E001801E102D05707CFD7A9
:02037A0012006F
:10037C007A0E01013D6F020E3E6F5A0E3F6F010E59
:10038C00406F440E396F050E3A6F000E3B6F000E36
:10039C003C6F560E356F050E366F000E376F000E24
:1003AC00386FFF0E446FFF0E456F000E466F000E48
:1003BC00476FAC8A900EAB6E948E949C9EAA03D021
:0803CC00AECF00F0FBD71200D8
:1003D40053C104F054C105F004C002F005C003F099
:1003E400044A052A55C100F056C101F00101554BDC
:1003F400562B00C0E9FF01C0EAFF02C0E1FF03C0C1
:10040400E2FFEECFE6FF02C0E9FF03C0EAFFEE52CF
:0E04140001E0E2D753C100F054C101F0120024
:10042200F1C05AF1F2C05BF10ADF00C054F1536B24
:1004320053510001F125E96E000E010153BFFF0E79
:100442000001F221EA6EEECF55F101014CA104D078
:1004520055C15AF111DF03D055C15AF152DE0101E3
:10046200532B800E5319006E800E5419005CE0E38A
:1004720015D025D0090E5A6FFFDE21D02C0E0101B6
:100482005A6FFADE1CD00D0E01015A6FF5DE17D03D
:1004920016D02A0E01015A6FEFDE11D001014C5124
:1004A200000AE7E04C51010AE5E04C51030AE6E09C
:1004B2004C51050AE8E04C51070AEAE0EAD712007B
:1004C200828482808294030E0B6E8A0E0C6E550E0D
:1004D2000D6E0D2EFED70C2EFCD70B2EFAD7000078
:1004E20000008284210E0101616FB4DD900E0101D2
:1004F200616FB0DD050E0101616FACDD130E01010C
:10050200616FA8DD200E0101616FA4DD210E0C6E6A
:10051200760E0D6E0D2EFED70C2EFCD700000C0EA3
:100522000101616F97DDBEDE410E0C6EEE0E0D6EA7
:100532000D2EFED70C2EFCD700005F6B606B99DD91
:020542001200A5
:10054400AECF43F1ABA202D0AB98AB8843C100F06D
:02055400120093
:0A055600000E9EBA010E006E1200A6
:100560000900F5CFE6FF0006FBE10106F9E1120004
:1005700081A201D0FDD781B201D0FDD781A201D0E7
:0E058000FDD7380E01015A6F8DDD14DE12001A
:10058E008196210E0C6E760E0D6E0D2EFED70C2E54
:10059E00FCD70000818A8184040E0C6E3D0E0D6E18
:1005AE000D2EFED70C2EFCD7000000008186040E07
:1005BE000C6E3D0E0D6E0D2EFED70C2EFCD70000D0
:1005CE0000008180040E0C6E3D0E0D6E0D2EFED7BA
:1005DE000C2EFCD700000000818A040E0C6E3D0E1E
:1005EE000D6E0D2EFED70C2EFCD700000000010E56
:1005FE000101536F000E546F800E006E800E541961
:10060E00005C02E15351050809E3100E5A6F43DDF9
:10061E00FF0E5A6F40DD534B542BEED7100E5A6F10
:10062E003ADD040E0C6E3D0E0D6E0D2EFED70C2E09
:10063E00FCD7000000005A6B2EDD040E0C6E3D0E32
:10064E000D6E0D2EFED70C2EFCD700000000100EE6
:10065E005A6F21DD040E0C6E3D0E0D6E0D2EFED763
:10066E000C2EFCD700000000440E5A6F14DD040E51
:10067E000C6E3D0E0D6E0D2EFED70C2EFCD700000F
:04068E000000120056
:100692000B6A0A6A096A00500402F4CF09F0F3CF28
:1006A20008F001500502F4CF0BF0F3CF0AF000502E
:1006B2000502F3500926F4500A22E86A0B2201507F
:1006C2000402F3500926F4500A22E86A0B2208C0F9
:1006D20000F009C001F00AC002F00BC003F01200E2
:1006E2000A0E01015A6FC8DD0D0E01015A6FC4DDF9
:0206F2001200F4
:1006F40053C104F054C105F004C0E9FF05C0EAFF8A
:10070400EE5203E0044A052AF7D704C002F005C0FC
:1007140003F0044A052A55C100F056C101F0010155
:10072400554B562B00C0E9FF01C0EAFF02C0E1FFB0
:1007340003C0E2FFEECFE6FF02C0E9FF03C0EAFF19
:10074400EE5201E0E2D753C100F054C101F01200AF
:100754000101566B030E565D0AE256515425E16EB3
:10076400000E5521E26E200EE66E562BF3D756513D
:100774005425E16E000E5521E26EE66A5607565185
:100784005425576F000E5521586F0A0E046E53C13D
:1007940000F078DD08C000F0300E002657C1E1FFFC
:1007A40058C1E2FF00C0E6FF0A0E046E53C100F018
:1007B40069DD00C053F10050000A01E102D0560780
:0407C400DED712006A
:1007C8009EA008D00101414B422BFF0ECF6EFF0EB9
:0607D800CE6E9E901100A0
:1007DE001DEC08F0816A120E936EF19E010E806E72
:1007EE00010E926E010EC26E8E0EC16E946AD56AA5
:1007FE000A0EAF6EAC84BBDD010E01014C6F6ADFD9
:10080E0001014C6B57DE020E0B6E450E0C6EA90EDF
:10081E000D6E0D2EFED70C2EFCD70B2EFAD7000028
:10082E00000001015F6B606B1EDCF1C053F1F2C082
:10083E0054F1A30E0101556F000E566FC4DD00C0BA
:10084E00F1F001C0F2F0E6DD819E01015F6B606B9D
:10085E000ADCF1C053F1F2C054F1920E0101556F52
:10086E00000E566FB0DD00C0F1F001C0F2F0D2DD27
:10087E0001015F6B010E606F3AEC00F0F1C053F1B5
:10088E00F2C054F1810E0101556F000E566F9BDDC3
:10089E0000C0F1F001C0F2F0BDDD01015F6B020E90
:1008AE00606F3AEC00F0F1C053F1F2C054F1D60E85
:1008BE000101556F000E566F86DD00C0F1F001C0CC
:1008CE00F2F0A8DD01015F6B030E606F3AEC00F0F1
:1008DE00F1C053F1F2C054F1C50E0101556F000E77
:1008EE00566F71DD00C0F1F001C0F2F093DD010131
:1008FE005F6B040E606F3AEC00F0F1C053F1F2C082
:10090E0054F1B40E0101556F000E566F5CDD00C040
:10091E00F1F001C0F2F07EDD01015F6B050E606F3C
:10092E003AEC00F0F1C053F1F2C054F1700E010137
:10093E00556F000E566F47DD00C0F1F001C0F2F0AA
:10094E0069DD01015F6B060E606F3AEC00F0F1C0DD
:10095E0053F1F2C054F1370E0101556F000E566F70
:10096E0032DD00C0F1F001C0F2F054DD01015F6B29
:10097E00070E606F3AEC00F0F1C053F1F2C054F183
:10098E00260E0101556F000E566F1DDD00C0F1F0F1
:10099E0001C0F2F03FDD1A0E0B6E5E0E0C6E6E0E87
:1009AE000D6E0D2EFED70C2EFCD70B2EFAD7000097
:1009BE00010E01014C6F8EDEE3DDF1C053F1F2C08A
:1009CE0054F1150E556F000E566FFDDC00C0F1F0A0
:1009DE0001C0F2F01FDD7EDEF1C053F1F2C054F122
:1009EE00480E0101556F000E566FEDDC00C0F1F0A0
:1009FE0001C0F2F00FDD6EDE010E01014C6F326BA5
:100A0E00336B000E335D02E1080E325D3DE232C102
:100A1E0000F033C101F0003600900136120E0024B2
:100A2E00516F010E0120526F32C100F033C101F03F
:100A3E00B20E046E0C0E056E25DE0D0E0026020E95
:100A4E00012251C1E1FF52C1E2FF00C0E6FF01C029
:100A5E00E6FF32C100F033C101F0003600900136DE
:100A6E00120E0024E96E010E0120EA6EEECF53F154
:100A7E00EECF54F1F1C055F1F2C056F12FDCCADCC5
:100A8E000101324B332BBDD725DE0D0E0B6EAF0E93
:100A9E000C6EB60E0D6E0D2EFED70C2EFCD70B2E39
:100AAE00FAD700000101326B336B346B4D6B4E6B1A
:100ABE00010E486F53EC01F0808801014D4B4E2B17
:100ACE00070E4C6F5DDDF1C053F1F2C054F1EB0E29
:100ADE00556F000E566F77DC00C0F1F001C0F2F0DA
:100AEE004DC153F14EC154F1E9C055F1EAC056F172
:100AFE0075EC01F04F6B506B000E505D02E1050E70
:100B0E004F5D1EE24F510001E925E96E0101505182
:100B1E000001EA21EA6EEECF01F00150200A0CE14D
:100B2E0001014F510001E925E16E01015051000113
:100B3E00EA21E26E300EE66E01014F4B502BDCD7F0
:100B4E00F1C053F1F2C054F1E9C055F1EAC056F1CB
:100B5E00CADD60DC070E01014C6F326B336B5F6BCD
:100B6E00606B3AEC00F080A802D0899801D0898899
:100B7E00070E01013215026E02C000F00036009021
:100B8E0000C04BF100C080FF8998020E0B6E960ECE
:100B9E000C6ED50E0D6E0D2EFED70C2EFCD70B2E19
:100BAE00FAD748A512D032C100F033C101F0003699
:100BBE0000900136120E0024E96E010E0120EA6E3D
:100BCE00EECF49F1EECF4AF105D0CBDC00C049F1B2
:100BDE0001C04AF149C153F14AC154F1F1C055F176
:100BEE00F2C056F175EC01F04F6B506B000E505D7C
:100BFE0002E1050E4F5D1EE24F510001F125E96E37
:100C0E00010150510001F221EA6EEECF01F00150C8
:100C1E00200A0CE101014F510001F125E16E0101A5
:100C2E0050510001F221E26E300EE66E01014F4B83
:100C3E00502BDCD711EC02F0E9C053F1EAC054F1AD
:100C4E00F1C055F1F2C056F1EAEC01F0000E335D41
:100C5E0002E1080E325D05E25F6B32C160F13AECE3
:100C6E0000F001014C6BF1C053F1F2C054F1EF0EE4
:100C7E00556F000E566FEAEC01F032C153F1E9C028
:100C8E0054F1EAC055F15FDDF1C053F1F2C054F1F9
:100C9E00E9C055F1EAC056F126DD11EC02F0F1C0C3
:100CAE0053F1F2C054F1E70E0101556F000E566F6D
:100CBE00EAEC01F049C153F14AC154F1E9C055F1D2
:100CCE00EAC056F175EC01F0F1C053F1F2C054F1E7
:100CDE00E9C055F1EAC056F106DD11EC02F0070E3F
:100CEE0001014C6F324B332B000E335D02E1080EC7
:100CFE00325DD8A03DD70A0E5A6F3DEC01F081BE91
:100D0E0002D0818E01D0819E1FDC0050010A1DE1B0
:100D1E0012DC00C034F10CD00101487114D04873BC
:100D2E0012D0487510D02A0E5A6F3DEC01F00BD040
:100D3E0001013451310AF0E03451320AF0E03451FD
:0E0D4E00330AEFE0F0D70101346BB7D6FFD7C0
:10103A0010EE15F0FD0E006E010E016E3C0EF66EFE
:0E104A000F0EF76E000EF86EB0EC02F0120002
:100D5C00000000000000005F000000070007001406
:100D6C007F147F14242A7F2A1223130864623649C5
:100D7C005522500005030000001C224100004122B6
:100D8C001C0014083E081408083E080800503000E7
:100D9C000008080808080060600000201008040221
:100DAC003E5149453E00427F400042615149462137
:100DBC0041454B311814127F1027454545393C4AA3
:100DCC0049493001710905033649494936064949F3
:100DDC00291E003636000000563600000814224149
:100DEC0000141414141400412214080201510906B1
:100DFC00324979413E7E1111117E7F494949363E77
:100E0C00414141227F4141221C7F494949417F098F
:100E1C000909013E4149497A7F0808087F00417F52
:100E2C0041002040413F017F081422417F40404057
:100E3C00407F020C027F7F0408107F3E4141413EFF
:100E4C007F090909063E4151215E7F091929464651
:100E5C004949493101017F01013F4040403F1F207A
:100E6C0040201F3F4038403F63140814630708704C
:100E7C0008076151494543007F41410002040810B5
:100E8C00200041417F0004020102044040404040E8
:100E9C00000102040020545454787F4844443838EC
:100EAC0044444420384444487F3854545418087EF1
:100EBC000901020C5252523E7F0804047800447D12
:100ECC0040002040443D007F1028440000417F40FA
:100EDC00007C041804787C080404783844444438B2
:100EEC007C14141408081414187C7C080404084896
:100EFC0054545420043F4440203C4040207C1C204F
:100F0C0040201C3C4030403C44281028440C50509D
:100F1C00503C4464544C44000836410000007F00AF
:100F2C000000413608001008081008784641467841
:100F3C00382056616C657572732031366269747332
:010F4C0000A4
:100F4D00332053696D756C2041443737313520207E
:010F5D000093
:100F5E00322061666669636820414443204348300D
:010F6E000082
:100F6F004D656E75206166666963686167653A20D5
:100F7F0031203D204E422020323D2043483020205A
:080F8F00333D53696D756C00E0
:100F97003120616666696368204EB07472616D6561
:010FA7000049
:100FA8003820766F69657320313620626974732042
:010FB8000038
:100FB90056657273696F6E2031362F30352F313097
:010FC9000027
:100FCA004144373731355F6E6F6B69615F3138463F
:010FDA000016
:100FDB002D2D2D204D454E55202D2D2D2D2D2D2DCF
:010FEB000005
:100FEC00557365732043443430353120382D3E31F0
:010FFC0000F4
:100FFD0041444320434830203130626974732020CE
:01100D0000E2
:02100E003D00A3
:02101000F300EB
:041012004E623D00ED
:02101600560082
:02101800FA00DC
:07101A00313233343536009A
:10102100313233343536373839303132333435367D
:081031003738393031322E004E
:020000040030CA
:0D00010022090EFF0081FF0FC007E00F4035
:00000001FF
